:020000020000FC
:100000004BC8189518951895189518951895189522
:100010001FC3189518951CC018951895A1C7189559
:100020001895189518950AFF061428071E9D012893
:100030006707329D013C9D01469D015065075A6945
:10004000070000005300440100007400D000FA11C2
:100050004A92BA93AA939A938A93FA93EA933A921A
:100060002A921A920A927A936A935A934A933A93EB
:100070002A931A930A934FB680E090E03798A4E44D
:10008000B1E00C910F710A9549F00A9571F00A954B
:1000900099F0025011F1025181F17EC004B115B105
:1000A000FD010483158302E078C004B115B1FD01A0
:1000B0000283138303E071C024B135B104E092D010
:1000C000FD0100871187003311410C9110F40F7B63
:1000D00001C000640C9305E060C004B115B1FD01DE
:1000E0000683178324B135B140E050E0ECD77AD0D5
:1000F000FD010287138707E150C004B115B112302A
:10010000C0F000E014E024B135B1021B130BFD0177
:10011000218122952F7030E0200F311F40E050E008
:10012000D2D793D0119501951040FD010487158712
:1001300014C004B115B1012B69F024B135B1FD0132
:10014000018102950F70201B304040E050E0BBD78A
:100150007CD0EBCFFD018487858724853585008D94
:100160000370000FE00FF81F26873787FD01008D11
:100170000395008F3E9604E021913191820F931FE9
:100180000A95D1F78C0144E050E0E1D7FD01068BE0
:10019000178B0C9100620C9301E01C91107E0F7183
:1001A000012B0C930F71005C07B91F980C91007A1A
:1001B000003A19F006B1006C06B94FBE09911991C9
:1001C00029913991499159916991799109901990A1
:1001D00029903990E991F99189919991A991B991D1
:1001E000499018952A2EBC01A02FC9010330A901FE
:1001F000A1F40DE110E077D7369527953695279530
:10020000200D311D9695879596958795969587959E
:1002100096958795820F931F14C007E210E063D76D
:1002200096958795969587959695879596958795B2
:10023000800D911DA33028F48C0143E04A1B69D73F
:10024000C8018C01CB01A22D08952A2EBC01A02F3C
:10025000C9010330A901A9F405E110E044D736959E
:100260002795369527953695279536952795021B20
:10027000130B880F892F881F90E0991F800F911F03
:100280001AC00CE110E02FD798018C011695079544
:100290001695079516950795201B310B8C0145E0A7
:1002A00038D7C801820F931FA33028F48C0143E094
:1002B0004A1B2FD7C8018C01CB01A22D0895FFCF77
:1002C000F894E4E4F1E000810F7700830AB3097049
:1002D0000ABB0BB309700BBB03E407B900E003B919
:1002E00007EC06B9349BFECF349A2181207F04B1FC
:1002F00015B10F70022B018316E517B917EC16B96B
:10030000349BFECF349A0F7024B135B12295207FF3
:10031000202B21830081007C0160008301E407B968
:1003200000E0068B078B3E9624E0019301932A950B
:10033000E1F70FEC06B97894FFCF009184010E51DC
:1003400049F0045149F10A5009F44AC00A5009F42D
:100350005EC077C0E1E6F1E0048115814AE050E03B
:10036000DED6EFE7F1E00283138302E30483EEE6D7
:10037000F1E0008308EB1BE00383148305E010E049
:100380000187128703E2078310871787108B24D118
:1003900040E010E022E037C021E631E0F9010481BD
:1003A0001581EFE7F1E0028313830CE30483EEE6AB
:1003B000F1E00BE1008300EC12E1038314830DE212
:1003C00010E00183128302E30783108701E00387B3
:1003D00014871587168740E0F9012085318515C0FF
:1003E000E1E6F1E0048115814AE050E098D6EFE7BC
:1003F000F1E00283138306E404830AE100936E01B3
:1004000040E010E02EE130E001E0E9D596C3D9D01C
:10041000E1E6F1E000810260008300916D0110E0EF
:100420000F5F1F4F42E050E092D621E030E0240FF2
:10043000351FA90148D6017011F004E1089508E2C2
:1004400008950AE0089500951AB310231ABB1BB350
:1004500010231BBB0CEB13E001501040E9F700C068
:1004600008951FB7F8942AB3202B2ABB00952BB30D
:1004700020232BBB2BE02A95F1F700C02AB32023C1
:100480002ABB2BB320232BBB06EA0A95F1F7000009
:100490001FBF08951FB7F8942AB3202B2ABB0095DD
:1004A0002BB320232BBB2BE92A95F1F700C02AB3ED
:1004B00020232ABB2BB320232BBB06E10A95F1F79F
:1004C00000001FBF08952FB7F8941AB3102B1ABB62
:1004D000102F10953BB331233BBB3BE03A95F1F72E
:1004E00000C03AB331233ABB3BB331233BBB13E1EA
:1004F0001A95F1F700C019B310230EE80A95F1F729
:1005000000002FBF012F08952FB7F8941AB3102BB6
:100510001ABB102F10953BB331233BBB4CEB53E080
:1005200041505040E9F700C03AB331233ABB3BB3E6
:1005300031233BBB16EB1A95F1F7000019B3109568
:10054000012340E353E041505040E9F700C02FBF82
:100550000895AA939A938A93A02F912F88E0A0FBE5
:10056000092F16F47EDF01C095DFA6958A95B9F7AD
:1005700089919991A9910895AA939A938A93A02F0A
:1005800090E088E096950A2F9EDF002309F090689E
:100590008A95C1F7092F89919991A991089538E019
:1005A000212F2170402F4170422711F4169504C06D
:1005B00028E112271695106806953A9589F7012FBC
:1005C000089500E00CBD09BD00BF0FBD07BD06BD0D
:1005D0000BBD0ABD04BD089501E200BF00E00FBDE0
:1005E00000B7007F07BD00E006BD00B90DBD0CE0FF
:1005F0000CBD0FEF0BBD00E00ABD04BDBB9A02E0CD
:1006000009BD41E010E020E030E0E9D402E0D3D4BD
:100610000023E1F709B500FFFDCF09B5046009BD6E
:100620000FB501600FBD08950CB50F3F29F00CB553
:1006300003950CBD01E0089500E008950CB500237A
:1006400029F00CB50A950CBD01E0089500E008956D
:100650008A93FA93EA933A922A921A920A927A9396
:100660006A935A934A933A932A931A930A938FB7A9
:1006700000E0A1D4002331F4EDE5F1E002810F7335
:100680000064028340E011E020E030E000E0A7D405
:1006900000E40EB9EDE5F1E003810460038312810B
:1006A000012F000F001F001F0370015029F00A9551
:1006B00001F10A9531F172C00FB10083002309F4F2
:1006C0006DC006FF03C003810E7F02C0038101607D
:1006D0000383008107FF03C00381026002C003811E
:1006E0000D7F038300810F73006802830CEC83D0BD
:1006F00055C00FB100830183012F006C02830BEB07
:10070000F6CF212F107C022F0A950F73012B028345
:100710002F7309F440C02181138110FF2EC02A9548
:1007200049F02A9571F02A9591F02A95B1F02A9511
:10073000E1F021C00F7310E0F801EC5BFE4F008187
:10074000D6CF0F7310E0F801E359FE4FF8CF0F73C7
:1007500010E0F801EF59FE4FF2CF0F7310E041E0C7
:1007600050E0400F511FAFD4C2CF0F7310E0F8011B
:10077000E957FE4FE4CF00E0BACF1FB110832450F9
:1007800069F4212F0F7310E041E050E0400F511F3A
:10079000022FA5D403C00F73006402838FBF099199
:1007A00019912991399149915991699179910990BA
:1007B000199029903990E991F99189911895F894B7
:1007C000B99A17B31A7F17BB18B3156018BB000F7F
:1007D000000F08650DB9EDE5F1E000E0008303814D
:1007E0000C7F038300E4028300E001830381037F25
:1007F0000383789408951EB11F70EDE5F1E029F0B0
:1008000003810860038300E008951381137F13833D
:100810000FB901E00895BA93AA938A9381E0E1E6C3
:10082000F1E0A481B58110D0002309F480E0E1E675
:10083000F1E004811581A017B10709F080E0082FCD
:100840008991A991B9910895BA93AA939A938A9399
:10085000A1E6B1E00C910C7F04600C9300E0FD0177
:10086000018302830483058306830783008701874E
:10087000028703871ED1DBD0102F117010FB0C9163
:1008800004F90C93E4E4F1E002851385003629E0D5
:10089000120718F00C910B7F0C930285023D1F404C
:1008A00018F00C9102600C930CB5002319F40C9114
:1008B00002FF08C00CB5002351F08689978981306A
:1008C00090402CF00C9101600C9301E004C00C915D
:1008D0000B7F0C9300E01C9114FF00E0899199912B
:1008E000A991B99108958A927A926A925A924A92FB
:1008F000BA93AA939A938A9390E0A3E0B0E0772406
:1009000001E002DE013009F055C011E003E321DE11
:1009100001E032DE502E10E042DE802F06E0402E55
:1009200001E02ADE182F3BDE802F4A94C9F701E050
:1009300023DE182F34DE0023E9F550926201009186
:1009400062010930B9F5492E429400EF4022440C6F
:1009500011E003ECFEDD11E0042DFBDD11E000E011
:10096000F8DD10E003EC1BDE102F042D18DE102F35
:1009700000E015DE802F01E0FFDD182F10DE0023E0
:10098000C9F480E02D0100E2602E01E0F5DD802E4B
:10099000182F05DE802F082DA201A1D301E0400E03
:1009A000571C6A9491F7E8DD182FF9DD002311F444
:1009B000739408C0AD0110E200E091D34F5F5F4F28
:1009C0001A95D1F793959096943008F498CF072D07
:1009D00089919991A991B99149905990699079908B
:1009E000899008958A93802F44E610E020E030E05B
:1009F00002E0F5D280936D0101E010E0482F4C5FDA
:100A000082D318B3102B18BB01E010E045E0481B5F
:100A10007AD3009518B3102318BB02E0CCD2002380
:100A2000E1F78991089508B30F7C08BB08953B2F27
:100A30002A2E40E0E0EDF0E024E001E611E0A6E43B
:100A4000B1E06D917C910080118060157105F0F02E
:100A50000280138006161706C8F046815781D80118
:100A600014964D935C9340855185D80116964D930D
:100A70005C9342855385D80118964D935C934485C9
:100A80005585D8011A964D935C9341E03E962A9580
:100A9000B1F6442351F420E0F80124832583268312
:100AA00027832087218722872387042FA22DB32F16
:100AB0000895BA933A2E282E00E080E0A1E6B1E036
:100AC000482F50E09A01440F551F420F531F28E052
:100AD00031E0240F351FE4E4F1E044815581F90150
:100AE0006081718146175707D0F0082F000F000F63
:100AF000FD010283F9014281FD0143830091480118
:100B0000152FF90120813181021B130B000F111FDA
:100B100050E005D3FD011281101B128301E0839583
:100B2000843110F4002361F2002319F400E50093EE
:100B30006301822DA32DB99108955A924A92BA93D6
:100B4000AA939A938A9355244424B9DB00916D01AA
:100B500010E041E050E0400F511FB5D2047031F079
:100B6000442443947BD200E00CBD25C0442011F006
:100B7000442477D2E4E4F1E00689178911234AF08E
:100B8000A1E8B1E0ED91FC91CF0103970817190797
:100B900058F44ADD002379F404E09FD10AE500937C
:100BA00083015524539407C03396E017F10718F4D6
:100BB00045DD002389F30DD0002311F4552029F2DF
:100BC0000091830189919991A991B9914990599086
:100BD00008959A928A927A926A925A924A92BA9313
:100BE000AA939A938A9377246ADB6624639484E4B5
:100BF00091E001E6402E01E0502EAEE6B1E00C910E
:100C0000062109F47CC0062D0A9551F00A9509F1D8
:100C1000025051F1045079F1085009F453C06FC0EB
:100C2000FD0105851685FC01228533850217130712
:100C300020F4FD012587368762C0021B130BFD01DE
:100C4000218132810217130708F459C07724739465
:100C500056C0FC0102851385FD01238134810217F2
:100C6000130708F44CC0F2CFFD0105811681FC0189
:100C700026893789F4CFFC0104811581FD01878421
:100C800090888016910668F4FC0104811581FD01AD
:100C90000787108B40E01EE120E030E003E09FD1A9
:100CA0002EC0801A910AF201438150E0FD010385B4
:100CB000148519D28014910410F103E07CD1002333
:100CC00029F6E2CF01E077D10023C9F477247394A9
:100CD0000C9105FF14C075DC00916D0110E041E03E
:100CE00050E0400F511FEFD10E7FF9D1F20100818A
:100CF0000860008300E1F1D00AE5FD01058B660C78
:100D000009F07DCFE1E6F1E00281FD012185328528
:100D1000102F110F110B2017310744F4102F110F52
:100D2000110B278130850217130740F04ADC08E0D9
:100D3000D4D00AE5FD01058B772473946CDD002384
:100D400031F43FDC0AE0FD01058B772473940091B8
:100D5000440106FD06C035DC08E2FD01058B772461
:100D60007394072D89919991A991B99149905990BE
:100D7000699079908990999008959A938A932AE03E
:100D80002093840180E090E000E006C01A3019F45E
:100D90003196859194910395402F50E0BA01440F0C
:100DA000551F460F571FE6E2F0E0E40FF51F1491C0
:100DB000112361F700E08030900719F0FC010995DC
:100DC000202F009184012017A9F32093840100E0D3
:100DD000402F50E0BA01440F551F460F571FE6E25F
:100DE000F0E0E40FF51F1491112321F330918401F9
:100DF000131719F43196859194910395E9CF8A934D
:100E0000F89400E808BD00E008BD01E01CDB43E009
:100E100050E010E800E063D14F5F5F4F1A95D1F7C3
:100E200000E307BB00DE00E0CADC4ADA1DD180E047
:100E3000082FD8DD44DA08DD83958230C8F3F3DD6E
:100E400000E000936D010093850104E1899108950C
:100E5000BA93AA939A938A9349D0002311F40AE58E
:100E60002FC081E090E0AC012ED1017079F4AC018B
:100E70004F5F5F4F28D1017049F4E5E8F1E0008150
:100E800002600083009184010183E9CFA0E0B0E01B
:100E9000AC014A0F5B1F17D1017069F00A2FA2DD68
:100EA0000EDAD2DC002339F00091610101FD03C0AC
:100EB0001ADD0EE105C0A395A23048F3B4DD08E2C7
:100EC00089919991A991B991089504E10895F7D96B
:100ED000FFCF77DBA8DDF3D9FFCFE5E8F1E01081A4
:100EE000102B10830091840101830895BA93AA9373
:100EF0009ADD72DB40E011E020E030E002E06FD0EC
:100F0000A4E4B1E010C01C960D911C911D97BCD0BB
:100F1000053610407CF488DB002361F0D0D902E074
:100F20004AD0002339F016960D911C9117970F3F68
:100F3000134019F446DB00E010C018960D911D9186
:100F4000085512402D913C911B97021B130B9CD00E
:100F5000043F1140C4F635DB01E0A991B991089531
:100F6000FA93EA937A936A935A934A931A930A9359
:100F70001FB7E7E8F1E004E04081518162817381AD
:100F8000452B462B472B49F0408141505040604053
:100F90007040408351836283738334960A950023A3
:100FA00059F71FBF09911991499159916991799107
:100FB000E991F991189510E0000F111F000F111F12
:100FC000F801E957FE4F0081118122813381012B05
:100FD000022B032B11F001E0089500E008958A929E
:100FE0006A925A924A92BA93AA939A938A93402EFB
:100FF000812E642EA90160E070E000E61AEE20E088
:1010000030E0B8D0C801D901482D50E060E070E070
:1010100008EE13E020E030E0ADD0080F191F2A1FC2
:101020003B1F462D50E060E070E0400F511F621FF3
:10103000731F5524440C551C440C551CF201E957F0
:10104000FE4F408351836283738389919991A99163
:10105000B9914990599069908990089500E003BF33
:10106000089503E003BF08950DE703BB00E002BB52
:1010700001E005BB03E003BF09B7006109BF789435
:10108000089500008895FECF11231AF4119501955B
:1010900010409801890108950FEC0DBF00E00EBFCC
:1010A000C0EAD0E080D0002309F08DD066DEE9DF11
:1010B000E8CFE199FECF08954F5F5F4FFADF4EBB57
:1010C0005FBBE09A0895FADF0DB308954F5F5F4F5D
:1010D0004EBB5FBBF894E29AE19A0FBE08950FB63B
:1010E000E8DF0DBBF5CF002411240030010741F0EB
:1010F0001695079510F4040E151E440F551FF5CFD5
:10110000002D112D08954A951AF0000F111FFBCFE5
:1011100008954A951AF016950795FBCF0895002477
:101120001124EFE0001F111F001C111C04161506EE
:1011300010F0041A150AEA95AAF7001F111FA00162
:101140000095109508955195419550400895FF27B9
:10115000552312F4F160F7DF112312F4F09506D055
:10116000DEDFF0FD03D0F1FDEECF0895119501957E
:1011700010400895002411241001E02FE12BE22BF0
:10118000E32B71F0369527951795079520F4040EFB
:10119000151E261E371E440F551F661F771FEDCFE5
:1011A00080019101089501E0089520E006D0E9F75B
:1011B0000895259102D0E9F708952D93015010402C
:1011C000202F212B089584E490E0FC0105911491D7
:1011D000FC013296A591B491FC013496259134918D
:1011E000422F432B19F0F901E4DF01C0DEDF069640
:1011F00010E08035910748F308952E0293023C0FCA
:10120000260204012C010A00E8024B03901AEE02A8
:1012100068012C010E006503BE031027E803DB0103
:101220002C01130049048104C05DD007DB01A40137
:101230002600EA0317B9031986031A51031B1C037E
:101240001BE6021BB1021A7D021A4B02191B02187F
:10125000EE0116C301159C011377011255011136D9
:0E126000010F1A010E00010DE9000BD4000A67
:0400000300000000F9
:00000001FF
